:100000000C9443050C948A050C948A050C948A057B
:100010000C948A050C948A050C948A050C948A0524
:100020000C948A050C948A050C94A90C0C947B0DF5
:100030000C94731C0C948A050C948A050C948A0504
:100040000C948A050C948A050C948A050C948A05F4
:100050000C948A050C94E71C0C948A050C948A0570
:100060000C948A050C948A050C948A050C948A05D4
:100070000C948A050C948A050C948A050C948A05C4
:100080000C948A050C948A050C948A050C948A05B4
:100090000C948A050C948A050C948A050C948A05A4
:1000A0000C948A050C948A050C948A05E80D0A0EB6
:1000B000F80E0A0EF80E4F0E720EF80EC70EDA0E7C
:1000C00002120212311231128F12CD12E714E7140C
:1000D000E612E714E713E713BB14E714E714D2148E
:1000E000141A082B1518171C12132F0C3080314CC2
:1000F0001E1F20352124222326272D252E802A4924
:10010000807B7A788080802C7E807C807F51504FED
:10011000801D1B7906111905363738107D528080F5
:1001200004160739090D0A0B0F33340E808028801E
:1001300080808080808080808080808080808080BF
:1001400080808080808080808080808080808080AF
:10015000808080808080808080808080808080809F
:100160004B6579626F6172642073746172742E0AD8
:100170000055534220636F6E666967757265642E21
:100180000A000D0A696E69740A005B445D005B43F6
:100190005D002C034600430036003600300043006B
:1001A000200041006C007400200043006F006E00CE
:1001B000740072006F006C006C006500720000003B
:1001C0000A0354004D004B002E00000004030904F4
:1001D00009028D00050100A032090400000103019D
:1001E00001000921110100012240000705810308D7
:1001F000000A0904010001030102000921110100A4
:1002000001224D000705820308000A0904020001CB
:1002100003000000092111010001223600070583B7
:100220000308000A09040300020300000009211169
:1002300001000122220007058403200001070504B4
:10024000032000010904040001030000000921113A
:100250000100012239000705850320000112011069
:100260000100000008EDFE0C66000101020001051E
:10027000010906A101050719E029E71500250195E7
:100280000875018102050819012905950575019177
:10029000029501750391010507190029F71500253D
:1002A0000195F875018102C00631FF0974A10109A9
:1002B00075150026FF009520750881020976150046
:1002C00026FF00952075089102C005010980A10153
:1002D000850216810026B7001A81002AB700751022
:1002E00095018100C0050C0901A1018503160100DB
:1002F000269C021A01002A9C02751095018100C0FB
:1003000005010902A1010901A10005091901290539
:10031000150025019505750181029501750381017F
:100320000501093009311581257F9502750881067F
:1003300009381581257F950175088106050C0A3855
:10034000021581257F950175088106C0C005010948
:1003500006A101050719E029E71500250195087593
:10036000018102950175088101050819012905958A
:100370000575019102950175039101050719002981
:10038000FF150026FF00950675088100C0636F6E9B
:1003900073756D65723A20253034580A007379738D
:1003A00074656D3A20253034580A000A0025303231
:1003B0005820006B6579626F6172643A20004C4589
:1003C000443A20253032580A00253032583A202548
:1003D0003031366225730A00722F63203031323398
:1003E0003435363738394142434445460A0064655E
:1003F0006C5F6B65795F6269743A2063616E277424
:100400002064656C3A20253032580A006164645FCC
:100410006B65795F6269743A2063616E277420614D
:1004200064643A20253032580A004F6E6573686F55
:10043000743A2074696D656F75740A00290A002585
:1004400075002F002575005D28002564002000251B
:100450006400200025640020002564007C00253015
:100460003258006D6F7573656B6579205B62746ED1
:100470007C782079207620685D287265702F616312
:100480006C293A205B006D6B5F776865656C5F7403
:10049000696D655F746F5F6D6178203D2025640A2A
:1004A000006D6B5F776865656C5F6D61785F737019
:1004B000656564203D2025640A006D6B5F74696D7D
:1004C000655F746F5F6D6178203D2025640A006D63
:1004D0006B5F6D61785F7370656564203D20256496
:1004E0000A006D6B5F696E74657276616C203D20E9
:1004F00025640A006D6B5F64656C6179203D202581
:10050000640A006D6B5F776865656C5F74696D6523
:100510005F746F5F6D6178203D2025640A006D6B0C
:100520005F776865656C5F6D61785F737065656442
:10053000203D2025640A006D6B5F74696D655F74F2
:100540006F5F6D6178203D2025640A006D6B5F6DE3
:1005500061785F7370656564203D2025640A006DD5
:100560006B5F696E74657276616C203D2025640A4C
:10057000006D6B5F64656C6179203D2025640A0025
:100580000A00257500363A20776865656C5F7469E6
:100590006D655F746F5F6D61783A20000A002575A4
:1005A00000353A20776865656C5F6D61785F7370C0
:1005B0006565643A20000A00257500343A207469A4
:1005C0006D655F746F5F6D61783A20000A00257574
:1005D00000333A206D61785F73706565643A20007E
:1005E0000A00257500323A20696E74657276616C76
:1005F000286D73293A20000A00257500313A2064DD
:10060000656C6179282A31306D73293A20000A0916
:100610002D2056616C756573202D0A004D3E004DEE
:1006200025643E20003F0073657420646566617533
:100630006C740A00433E200077686572652064652B
:100640006C74613A20637572736F723D25642C205F
:10065000776865656C3D25640A5365652068747428
:10066000703A2F2F656E2E77696B697065646961CA
:100670002E6F72672F77696B692F4D6F7573655F8A
:100680006B6579730A000A092D204D6F7573656BD0
:100690006579202D0A4553432F713A0971756974A4
:1006A0000A313A0964656C6179282A31306D732901
:1006B0000A323A09696E74657276616C286D732925
:1006C0000A333A096D61785F73706565640A343A7C
:1006D0000974696D655F746F5F6D61780A353A09F9
:1006E000776865656C5F6D61785F73706565640AD6
:1006F000363A09776865656C5F74696D655F746F1C
:100700005F6D61780A0A703A097072696E742076BA
:10071000616C7565730A643A097365742064656673
:1007200061756C74730A75703A092B310A646F77BE
:100730006E3A092D310A706775703A092B31300A0B
:100740007067646F776E3A092D31300A0A737065ED
:100750006564203D2064656C7461202A206D617899
:100760005F7370656564202A202872657065617406
:10077000202F2074696D655F746F5F6D6178290A41
:10078000003F004D3E2000433E20004C25640A00FF
:100790000A092D20436F6E736F6C65202D0A455337
:1007A000432F713A09717569740A6D3A096D6F7555
:1007B00073656B65790A000A092D204D61676963CD
:1007C000202D0A643A0964656275670A783A0964FB
:1007D00065627567206D61747269780A6B3A0964A5
:1007E00065627567206B6579626F6172640A6D3A44
:1007F000096465627567206D6F7573650A763A09DD
:1008000076657273696F6E0A733A097374617475F1
:10081000730A633A09636F6E736F6C65206D6F6462
:10082000650A302D343A096C61796572302D3428AF
:100830004631302D4634290A506175733A09626F8A
:100840006F746C6F616465720A6E3A094E4B524F59
:100850000A003F004E4B524F3A206F66660A004E28
:100860004B524F3A206F6E0A0074696D65725F7269
:10087000656164333228293A202530346C580A00E7
:100880006B6579626F6172645F6E6B726F3A20257F
:10089000580A006B6579626F6172645F69646C65A8
:1008A0003A2025580A006B6579626F6172645F7047
:1008B000726F746F636F6C3A2025580A00686F730B
:1008C000745F6B6579626F6172645F6C65647328D5
:1008D000293A2025580A000A092D2053746174759D
:1008E00073202D0A004743433A20342E392E3220FC
:1008F0004156522D4C4942433A20312E382E307306
:10090000766E204156525F415243483A20617672DA
:10091000350A004F5054494F4E533A204C554641EA
:10092000204D4F5553454B45592045585452414B46
:10093000455920434F4E534F4C4520434F4D4D4159
:100940004E44204E4B524F204B45594D41505F5322
:10095000454354494F4E20343039360A00425549F8
:100960004C443A20386361623765362D646972748D
:1009700079202831383A31353A3130204D617920AB
:1009800033312032303137290A005649443A203079
:10099000784645454428544D4B2E29205049443A29
:1009A00020307836363043284643363630432041AF
:1009B0006C7420436F6E74726F6C6C657229205674
:1009C00045523A203078303130300A0044455343A4
:1009D0003A20544D4B2E206B6579626F6172642012
:1009E0006669726D7761726520666F722046433664
:1009F0003630430A000A092D2056657273696F6EFE
:100A0000202D0A000A6D6F7573653A206F66660ABD
:100A1000000A6D6F7573653A206F6E0A000A6B6588
:100A200079626F6172643A206F66660A000A6B65CC
:100A300079626F6172643A206F6E0A000A6D6174A8
:100A40007269783A206F66660A000A6D617472698D
:100A5000783A206F6E0A000A64656275673A206F03
:100A60006E0A000A64656275673A206F66660A005E
:100A70000A0A626F6F746C6F616465722E2E2E208D
:100A800000433E20000011241FBECFEFDAE0DEBF9E
:100A9000CDBF04B603FE27C08091A2029091A302AD
:100AA000A091A402B091A5028730904BA740B04B13
:100AB000D1F41092A2021092A3021092A4021092FA
:100AC000A50214BE84B7877F84BF0FB6F894A8959B
:100AD00080916000886180936000109260000FBE7A
:100AE000E0E0F8E3099511E0A0E0B1E0E4EEFAE41B
:100AF00002C005900D92A833B107D9F722E0A8E310
:100B0000B1E001C01D92A23AB207E1F70E94D709F5
:100B10000C9470250C940000FF93EF93E091380142
:100B2000F0913901309709F00995EF91FF910895FF
:100B3000FC018591803011F0EFDFFBCF0895FF2796
:100B4000E0E230E247FF0CC0419597FF09C0EDE2BB
:100B50006095709580959095611D711D811D911D09
:100B600027FF02C0219530E350E2AA27660F771FC6
:100B7000881F991FAA1FA41710F0A41B63955A95EC
:100B8000A9F7AA3008F0A95FA05DAF93F3956115AE
:100B900071058105910541F7ED3211F4EF93F3955D
:100BA000F21718F43F93F395FBCF8F91B5DFFA95C9
:100BB000E1F70895E991F9918591803021F085322E
:100BC00019F0AADFF9CF089520E0E8945591553245
:100BD000C1F3503311F4689455915A3348F450538B
:100BE00090F3220F022E220F220F200D250FF4CF9B
:100BF0000EF4219589919991533619F3533729F1C0
:100C0000533559F1BC0188279927E8945C3621F4C3
:100C10008991999168945591543639F446EF7EF054
:100C200077FF0DC08FEF9FEF0AC055374AE039F0CC
:100C3000583540E121F0523642E009F00895FF9323
:100C4000EF937DDFEF91FF91B7CFFF93EF93FC011F
:100C500081918030B9F360DFFBCFFF93EF9368DFC2
:100C6000F1CFDF93CF93CDB7DEB72596A3DFCF913A
:100C7000DF91089561FF02C02D9808952D9A08957F
:100C800084B18F6184B93E98469A3F9A8AB1806F49
:100C90008AB95F9A479884B1806684B985B18066C5
:100CA00085B9EAE4F1E01192119281E0EA35F807A2
:100CB000D1F7EAE3F1E01192119281E0EA34F8070A
:100CC000D1F78AE491E090935D0180935C018AE31F
:100CD00091E090935B0180935A010895AF92BF9287
:100CE000DF92EF92FF920F931F93CF93DF93809148
:100CF0005A0190915B0120915C0130915D0130932C
:100D00005B0120935A0190935D0180935C0100E0A8
:100D100010E0C1E0D0E085B1982F907E03FF02C0C3
:100D200020E101C028E0802F8770892B822B85B9B4
:100D3000BE01002E02C0660F771F0A94E2F75B0126
:100D4000A094B09440E050E08BB18F7080689A011D
:100D500094E0220F331F9A95E1F7822B8BB92AE09A
:100D60002A95F1F700C0CA01880F991FA0915A0176
:100D7000B0915B01A80FB91F2D913C912623372319
:100D8000232B09F0479AE5E3EA95F1F70000D6B482
:100D90005F98FAE0FA95F1F700C0A0915C01B0917C
:100DA0005D017D01E80EF91EF701369B05C020812B
:100DB00031812A213B2104C020813181262B372B10
:100DC0003183208326B5ED2CF12C2D1518F026B596
:100DD00030E004C026B530E021503F4F2E193F09C6
:100DE0002630310568F020915A0130915B01280FBF
:100DF000391FF90120813181A80FB91F2D933C9330
:100E0000FAE1FA95F1F700C047985F9A8BE291E01A
:100E10000197F1F700C000004F5F5F4F4830510568
:100E200009F092CFA0915C01B0915D01E0915A016F
:100E3000F0915B0150962D913C9151978089918959
:100E40002817390751F00E94B11C60935E0170931E
:100E50005F0180936001909361010F5F1F4F00312C
:100E6000110509F058CF81E0DF91CF911F910F91CB
:100E7000FF90EF90DF90BF90AF90089520915C01BC
:100E800090915D01E22FF92FE80FF11DE80FF11DA0
:100E900080819181089581FF02C02E9808952E9A35
:100EA00008958091860108959FB7F8941092650186
:100EB0009FBF90919902943009F057C09091E9003A
:100EC0009F703091EC00232F217030FD20E8922B91
:100ED00024E02093E9002091EB0020FF43C0209103
:100EE000EE0027FF3FC020916201222321F02091D4
:100EF000E80025FF37C01092620126E03091E8003B
:100F000035FD15C030919902343061F53091EB0018
:100F100035FD28C0215021F481E08093620122C078
:100F2000EFE9FFE03197F1F700C00000E7CF8093D1
:100F3000F1008091E80085FD0AC08091E80080FF03
:100F4000FCCF8091E8008E778093E80006C08FB7D1
:100F5000F89421E0209365018FBF9F709093E90082
:100F600080E008959F709093E9008FEF0895CF93EC
:100F7000DF9300D01F92CDB7DEB79C01809199021C
:100F8000843019F593E099833B832A839093E90099
:100F90008FEF9091E800815095FD06C095ED9A95F0
:100FA000F1F700008111F5CF8091E80085FF0DC0B9
:100FB00040E050E063E070E0CE0101960E94990AA3
:100FC0008091E8008E778093E8000F900F900F904B
:100FD000DF91CF910895CF93DF9300D01F92CDB7CB
:100FE000DEB720919902243021F522E029839B83EA
:100FF0008A8383E08093E9008FEF9091E80081502D
:1010000095FD06C095ED9A95F1F700008111F5CF99
:101010008091E80085FF0DC040E050E063E070E0A3
:10102000CE0101960E94990A8091E8008E77809304
:10103000E8000F900F900F90DF91CF9108952091CD
:1010400099022430F1F422E02093E9002FEF30914F
:10105000E800215035FD06C035ED3A95F1F7000066
:101060002111F5CF2091E80025FF0BC040E050E0B2
:1010700065E070E00E94990A8091E8008E77809385
:10108000E8000895CF93DF9320919902243009F06E
:1010900048C0EC0180910A018823E1F080910B01A6
:1010A0008823C1F085E08093E9008FEF9091E800FC
:1010B000815095FD06C09AE29A95F1F700C0811122
:1010C000F5CF8091E80085FF2CC040E050E060E261
:1010D00070E017C081E08093E9008FEF9091E80005
:1010E000815095FD06C095ED9A95F1F700008111AC
:1010F000F5CF8091E80085FF14C040E050E068E043
:1011000070E0CE010E94990A8091E8008E7780936A
:10111000E80080E2FE01A6E6B1E001900D928A951A
:10112000E1F7DF91CF9108958EE891E00E94980554
:1011300080919802811109C00E942E0C0E948B0C94
:101140008091E20084608093E20008958AE891E053
:101150000E949805109298020895089520916301C5
:101160002F5F822F62E30E943625992319F0209386
:10117000630108951092630180916501882371F1E4
:1011800080919902843041F58091E9008F7020911F
:10119000EC00922F917020FD90E8892B94E09093C1
:1011A000E9009091EB0090FF14C09091EE0097FF42
:1011B00010C09091E80095FF03C01092F100F9CFA4
:1011C0009091E80090FF05C09091E8009E77909381
:1011D000E8008F708093E90010926501089542E065
:1011E00061EC81E00E94A80B42E061EC82E00E9489
:1011F000A80B42E061EC83E00E94A80B42E261ECA4
:1012000084E00E94A80B42E261EC85E00C94A80BFC
:1012100080919B02833009F455C030F4813071F025
:10122000823009F48EC008958A3009F47AC08B3078
:1012300009F460C0893009F09CC020C080919A02F6
:10124000813A09F096C08091E800877F8093E8009A
:1012500080919E0290919F02892B21F460E286E6A4
:1012600091E003C060E080E090E070E00E94E40A5A
:101270008091E8008B778093E800089580919A022E
:10128000813209F076C080919E0290919F02009772
:1012900019F0049709F06DC08091E800877F809372
:1012A000E8008091E80082FD05C0809199028111DB
:1012B000F8CF5FC08091F100809386018091E800B3
:1012C0008B7753C080919A02813A09F052C0809185
:1012D0009E0290919F02892B09F04BC08091E800FB
:1012E000877F8093E8008091E80080FFFCCF8091A9
:1012F0000A0136C080919A028132D9F580919E020E
:1013000090919F02892BA9F58091E800877F8093B7
:10131000E8000E94DD0B80919C0280930A010C94EE
:10132000091580919A02813221F58091E800877F2A
:101330008093E8000E94DD0B80919D0280938701DD
:10134000089580919A02813AA1F48091E800877F04
:101350008093E8008091E80080FFFCCF80918701B6
:101360008093F1008091E8008E778093E8000C94E0
:10137000DD0B08950895089580918601809364019E
:101380001092860180E00E944B070E94A4100C94EA
:1013900009150C94BC090E94311C80919702882386
:1013A00029F00E945A1C81110C94830A089584B775
:1013B000877F84BF0FB6F894A895809160008861FC
:1013C00080936000109260000FBE90E080E80FB63E
:1013D000F89480936100909361000FBE84E597E0DC
:1013E0000E94E91B82E891E00E9498050E94BA09D8
:1013F0000E94D10F0E942E0C0E948B0C8091E20063
:1014000084608093E2007894809199028430E1F7BF
:1014100081E791E00E9498050E94D30F80E091E05F
:101420000E94100F80E691E00E9498050E94BB097F
:1014300080919902853019F40E94CB09F9CF0E945E
:10144000D70FF6CF0E946F1C8091640180938601B4
:1014500008950C94220A292F332723303105C9F02F
:1014600064F42130310581F02230310509F043C0A8
:101470008DE890E020ED31E042C021323105F1F0FD
:101480002232310541F137C082E190E02DE532E0B2
:1014900036C099278130910541F08230910541F0A5
:1014A000892B49F5ECECF1E005C0E0ECF1E002C07D
:1014B000E2E9F1E0849190E09F0121C06530D8F429
:1014C000E62FF0E0EE0FFF1FED5DFE4F2081318132
:1014D00089E090E014C0653070F470E0FB01EE0F1D
:1014E000FF1FE75EFE4F20813181FB01EC5EFE4F66
:1014F000808190E004C080E090E020E030E0FA01DC
:1015000031832083089580E189BD82E189BD09B4DA
:1015100000FEFDCF8091D8008F7D8093D800809110
:10152000E00082608093E0008091E00081FDFCCFCC
:101530000895CF92DF92EF92FF920F931F93CF9374
:10154000DF93EC018B016A010E94FC0B811133C017
:10155000C114D10439F0F60180819181081B190B67
:10156000C80FD91FE12CF12C0115110519F180913B
:10157000E80085FD16C08091E8008E778093E80032
:10158000C114D10449F0F60180819181E80EF91E61
:10159000F182E08285E00FC00E94FC0B882321F3DA
:1015A0000AC089918093F10001501109FFEFEF1AF1
:1015B000FF0ADACF80E0DF91CF911F910F91FF906A
:1015C000EF90DF90CF9008952091A0023091A1027A
:1015D0002617370748F06115710539F42091E800A6
:1015E0002E772093E80001C0B90140E06115710534
:1015F000A9F120919902222309F443C0253009F46E
:1016000042C02091E80023FD40C02091E80022FD67
:1016100032C02091E80020FFE9CF4091F3002091F3
:10162000F20030E0342BFC01CF016115710559F057
:101630002830310540F481918093F10061507109A7
:101640002F5F3F4FF1CF41E02830310509F040E0F6
:101650002091E8002E772093E800C8CF4111C9CF30
:101660000AC080919902882361F0853061F08091F1
:10167000E80083FD0AC08091E80082FFF2CF80E09D
:10168000089582E0089583E0089581E0089520910F
:10169000A0023091A1022617370748F061157105A5
:1016A00039F42091E8002E772093E80001C0B901B9
:1016B000FC0120E06115710591F180919902882368
:1016C00009F440C0853009F43FC08091E80083FDF3
:1016D0003DC08091E80082FD2FC08091E80080FF2E
:1016E000E9CF2091F3008091F20090E0922B6115F8
:1016F000710559F08830910540F424912093F10050
:101700003196615071090196F2CF21E0089709F0F6
:1017100020E08091E8008E778093E800CBCF211104
:10172000CCCF0AC080919902882361F0853061F0A6
:101730008091E80083FD0AC08091E80082FFF2CF2B
:1017400080E0089582E0089583E0089581E008959F
:10175000982F973058F59093E900981739F07091C9
:10176000EC002091ED005091F00003C0242F762F63
:1017700050E021FF19C03091EB003E7F3093EB0029
:101780003091ED003D7F3093ED003091EB00316002
:101790003093EB007093EC002093ED005093F00039
:1017A0002091EE0027FF07C09F5FD3CF8F708093FB
:1017B000E90081E0089580E0089580919A0287FF12
:1017C00011C08091E80082FD05C0809199028111CD
:1017D000F8CF11C08091E8008B770BC080919902FF
:1017E000882349F08091E80080FFF8CF8091E800DD
:1017F0008E778093E80008952091E4003091E50011
:1018000095E64091EC00842F817040FF22C08091CA
:10181000E80080FD1CC080919902882391F08530FA
:1018200091F08091EB0085FD10C04091E400509153
:10183000E5004217530729F39A01915011F784E00C
:10184000089582E0089583E0089581E0089580E09E
:1018500008954091E80042FFDECF08950E949C0C5D
:101860000E94A40CE0EEF0E0808181608083E8EDCE
:10187000F0E080818F77808319BCA7EDB0E08C9178
:101880008E7F8C9380818F7E808310929802089542
:101890000F931F93CF93DF930E949C0C0E94A40C84
:1018A000C8EDD0E088818F778883888180688883BD
:1018B00088818F7D888319BC1092990210929502BD
:1018C000109297021092960200EE10E0F8018081CB
:1018D0008B7F808388818160888342E060E080E044
:1018E0000E94A80BE1EEF0E080818E7F8083E2EE23
:1018F000F0E0808181608083808188608083F8014E
:1019000080818E7F8083888180618883DF91CF9101
:101910001F910F910895E8EDF0E080818F7E808324
:10192000E7EDF0E080818160808384E082BF81E028
:10193000809398020C94480CE8EDF0E080818E7F53
:1019400080831092E20008951092DA001092E10074
:1019500008951F920F920FB60F9211242F933F9369
:101960004F935F936F937F938F939F93AF93BF93A7
:10197000EF93FF938091E10082FF0BC08091E20022
:1019800082FF07C08091E1008B7F8093E1000E947D
:10199000AE088091DA0080FF1FC08091D80080FFE0
:1019A0001BC08091DA008E7F8093DA008091D9008D
:1019B00080FF0DC080E189BD82E189BD09B400FED0
:1019C000FDCF81E0809399020E94940805C019BC64
:1019D000109299020E94A6088091E10080FF19C030
:1019E0008091E20080FF15C08091E2008E7F80939D
:1019F000E2008091E20080618093E2008091D80053
:101A000080628093D80019BC85E0809399020E947F
:101A1000C9098091E10084FF30C08091E20084FF19
:101A20002CC080E189BD82E189BD09B400FEFDCFF3
:101A30008091D8008F7D8093D8008091E1008F7EC7
:101A40008093E1008091E2008F7E8093E20080919C
:101A5000E20081608093E20080919502882311F07A
:101A600084E007C08091E30087FD02C081E001C0EF
:101A700083E0809399020E94290A8091E10083FF0C
:101A800029C08091E20083FF25C08091E100877F1B
:101A90008093E10082E080939902109295028091F8
:101AA000E1008E7F8093E1008091E2008E7F809341
:101AB000E2008091E20080618093E20042E060E019
:101AC00080E00E94A80B8091F00088608093F00075
:101AD0000E94AD08FF91EF91BF91AF919F918F91BF
:101AE0007F916F915F914F913F912F910F900FBE1A
:101AF0000F901F9018951F920F920FB60F921124FE
:101B00002F933F934F935F936F937F938F939F9305
:101B1000AF93BF93CF93DF93EF93FF93C091E9000F
:101B2000CF708091EC00D82FD17080FDD0E810925A
:101B3000E9008091F000877F8093F00078940E9404
:101B4000BF0D1092E9008091F00088608093F00052
:101B5000CD2BCF70C093E900FF91EF91DF91CF9132
:101B6000BF91AF919F918F917F916F915F914F91B5
:101B70003F912F910F900FBE0F901F9018951F93BC
:101B8000CF93DF93CDB7DEB7AA970FB6F894DEBF39
:101B90000FBECDBFEAE9F2E088E08E0F9091F10030
:101BA00091938E13FBCF0E9408098091E80083FF78
:101BB0001FC180919A0290919B02492F50E04A30B8
:101BC000510508F015C1FA01EA5AFF4F0C94562549
:101BD000803881F0823809F00BC180919E028F70AD
:101BE0008093E9008091EB0085FB882780F91092B3
:101BF000E90006C08091960290919702911182604F
:101C00009091E800977F9093E8008093F100109204
:101C1000F100C8C0282F2D7F09F0EAC0882319F0F1
:101C2000823061F0E5C080919C02813009F0E0C013
:101C3000933009F080E0809397022BC080919C0242
:101C4000811127C080919E028F7009F4D1C08093CA
:101C5000E9002091EB0020FF1CC0933021F480911B
:101C6000EB00806214C09091EB0090619093EB00C8
:101C700021E030E0A90102C0440F551F8A95E2F728
:101C80004093EA001092EA008091EB008860809314
:101C9000EB001092E9008091E800877F86C08111F7
:101CA000A7C010919C021F778091E3008078812B60
:101CB0008093E3008091E800877F8093E8000E9492
:101CC000DD0B8091E80080FFFCCF8091E30080680D
:101CD0008093E300111102C082E001C083E0809391
:101CE000990286C08058823008F082C080919C02A0
:101CF00090919D028C3D53E0950779F583E08A83AE
:101D00008AE289834FB7F894DE01139620E03EE023
:101D100051E2E32FF0E050935700E49120FF03C01D
:101D2000E295EF703F5FEF708E2F90E0EA3010F099
:101D3000C79601C0C0968D939D932F5F243149F7BC
:101D40004FBF8091E800877F8093E8006AE270E0EF
:101D5000CE0101960E94E40A14C0AE014F5F5F4FAE
:101D600060919E020E942B0ABC01892B09F440C09D
:101D70009091E800977F9093E80089819A810E9472
:101D8000470B8091E8008B778093E80031C0803862
:101D900079F58091E800877F8093E8008091950233
:101DA0008093F1008091E8008E778093E8000E9494
:101DB000DD0B1EC081111CC090919C029230C0F4BA
:101DC0008091E800877F8093E800909395020E94BD
:101DD000DD0B80919502811106C08091E30087FDA3
:101DE00002C081E001C084E0809399020E94EF0864
:101DF0008091E80083FF0AC08091E800877F80938C
:101E0000E8008091EB0080628093EB00AA960FB609
:101E1000F894DEBF0FBECDBFDF91CF911F91089523
:101E200090938D0180938C010895E0918C01F09145
:101E30008D01309721F00190F081E02D099480E030
:101E40000895EF92FF920F931F93CF93DF93E0914A
:101E50008C01F0918D013097B1F18C010280F381FA
:101E6000E02D09958091840282FF2DC080FF04C07F
:101E700083EB93E00E949805E80110E28DEAE82EDA
:101E800083E0F82E8091840280FF0BC088811F922E
:101E90008F93FF92EF920E9431060F900F900F9058
:101EA0000F90115021961111EDCF8091840280FF87
:101EB0000AC08BEA93E0DF91CF911F910F91FF90C1
:101EC000EF900C949805DF91CF911F910F91FF90A7
:101ED000EF900895E0918C01F0918D01309721F001
:101EE0000480F581E02D09940895CF93DF93EC01F0
:101EF00080918A0190918B01C817D90709F1D0937D
:101F00008B01C0938A01E0918C01F0918D01309793
:101F1000B9F00680F781E02DCE0109958091840209
:101F200082FF0EC080FF0CC0DF93CF938DE993E05A
:101F30009F938F930E9431060F900F900F900F90F8
:101F4000DF91CF910895CF93DF93EC0180918801C9
:101F500090918901C817D90709F1D0938901C093DD
:101F60008801E0918C01F0918D013097B9F00084E7
:101F7000F185E02DCE0109958091840282FF0EC08B
:101F800080FF0CC0DF93CF938DE893E09F938F93F6
:101F90000E9431060F900F900F900F90DF91CF911C
:101FA00008950C94A5100E949C1C0C9440065F920E
:101FB0006F927F928F929F92AF92BF92CF92DF9259
:101FC000EF92FF920F931F93CF93DF9300D000D037
:101FD0001F92CDB7DEB70E946E060FE811E0512CBC
:101FE00088248394912C852D0E943E075C01F80182
:101FF000C080D180C826D926C114D10439F45394A5
:102000000E5F1F4FF8E05F12EECF3FC08091840259
:1020100081FD0E94A610E12CF12C34010E2C02C08F
:10202000660C771C0A94E2F7C3018C219D21892B51
:1020300021F1E9825A8221E0C3018A219B21892B67
:1020400009F420E02B830E94A51C8160782F9D83DA
:102050008C8349815A816B818D810E94DC1049817A
:102060005A816B817C818D810E941F1CF8018081C7
:1020700091816826792671826082FFEFEF1AFF0A4C
:1020800080E1E816F10449F6BACF8FEF89838A839D
:102090001B820E94A51C8160782F9D838C834981BF
:1020A0005A816B818D810E94DC100E941E1C0E944F
:1020B000661F10918E010E94150F181771F10E9472
:1020C000150F80938E019091840292FF0EC090FFB5
:1020D0000CC01F928F938EEB93E09F938F930E947F
:1020E00031060F900F900F900F9080918E010F90FE
:1020F0000F900F900F900F90DF91CF911F910F9144
:10210000FF90EF90DF90CF90BF90AF909F908F9017
:102110007F906F905F900C942F1C0F900F900F90FA
:102120000F900F90DF91CF911F910F91FF90EF9043
:10213000DF90CF90BF90AF909F908F907F906F90E7
:102140005F9008950C944B0708950895EF92FF92C5
:102150000F931F93CF93DF9388ED93E00E94980530
:10216000C0E0D0E08DE2E82E81E0F82E09EC13E02B
:102170008C2F0E943E070E94041CFF92EF929F93B7
:102180008F93DF93CF931F930F930E943106219675
:102190008DB79EB708960FB6F8949EBF0FBE8DBF41
:1021A000C830D10529F7DF91CF911F910F91FF9092
:1021B000EF90089508950895CF93DF93CDB7DEB7DC
:1021C0002B970FB6F894DEBF0FBECDBF942F4F8371
:1021D000252F588769877A878B874A855B85452BAA
:1021E00021F02F3F09F59F3FF9F4DE01119686E0BB
:1021F000FD0111928A95E9F785E0FE01379601907D
:102200000D928A95E1F749815A816B817C818D819C
:102210009E810E94DC172B960FB6F894DEBF0FBE8E
:10222000CDBFDF91CF9108954F81588569857A851B
:102230008B850E941F1CD9CFCF93882309F465C0DA
:10224000C82F8CEF8C0F813A20F080E58C0F8E32F6
:1022500048F48C2F0E94B022811157C08C2F0E940D
:10226000A51A0CC080E28C0F883058F4C77081E04A
:1022700001C0880FCA95EAF70E94501BCF910C94B9
:10228000941B8BE58C0F833078F4C53A29F0C63A5D
:1022900031F083E890E005C081E890E002C082E878
:1022A00090E0CF910C94750F88E58C0F853168F51F
:1022B000C83A89F0C93A91F0CA3A99F0CB3AA1F0FC
:1022C000CC3AA9F0CD3AB1F0CE3AB9F0CF3AC1F05C
:1022D00080E090E017C082EE90E014C089EE90E0BC
:1022E00011C08AEE90E00EC085EB90E00BC086EB4B
:1022F00090E008C083EB90E005C084EB90E002C062
:1023000087EB90E0CF910C94A30FCF910895882391
:1023100049F19CEF980F913A20F090E5980F9E328A
:1023200018F40E94F81A0DC090E2980F983058F4F3
:10233000877091E001C0990F8A95EAF7892F0E9472
:10234000561B0C94941B9BE5980F933020F480E06F
:1023500090E00C94750F885A853120F480E090E06D
:102360000C94A30F0895882321F00E94501B0C9415
:10237000941B0895882321F00E94561B0C94941BF3
:102380000895BF92CF92DF92EF92FF920F931F9327
:10239000CF93DF9300D000D000D0CDB7DEB725E0DB
:1023A000FC01DE01119601900D922A95E1F7FC01E6
:1023B00040815181028163817481258122952F7032
:1023C0006115710509F403C35F3F19F44F3F09F428
:1023D000FEC26C01862F7D836C83602F782F8D81E8
:1023E0002E830E94381A182FB92E0E94371A0E9485
:1023F0002719EB2DE295EF70F0E0E05AFF4F2E81A8
:102400000C9456258B2D807F9B2D9F70F92E882351
:1024100019F0F29490EFF922002349F0FF2009F41B
:1024200083C28F2D0E94631B0E94941B7DC2812F4B
:102430000E948711FF2009F4CAC28F2D0E94691BD8
:1024400026960FB6F894DEBF0FBECDBFDF91CF91B9
:102450001F910F91FF90EF90DF90CF90BF900C9461
:10246000941B8B2D807F9B2D9F70F92E803219F04D
:10247000F29480EFF822112319F0113009F12AC0EB
:102480000023B1F08F2D222351F1213041F5269602
:102490000FB6F894DEBF0FBECDBFDF91CF911F9175
:1024A0000F91FF90EF90DF90CF90BF900C94731B33
:1024B000222319F0213009F48AC20E947C1B2DC00E
:1024C0000023F1F0263008F082C20E944D1B8F21BC
:1024D00029F023C00023F9F0211116C08F2D269674
:1024E0000FB6F894DEBF0FBECDBFDF91CF911F9125
:1024F0000F91FF90EF90DF90CF90BF900C94B311AD
:10250000253008F064C209C0F601858180FF0CC245
:102510008F708583E3CF21111CC28F2D83C12B2D9A
:1025200026952695237030E02115310521F02130C4
:102530003105D1F04CC2002321F0812F9B2D9370E7
:1025400002C080E090E026960FB6F894DEBF0FBE82
:10255000CDBFDF91CF911F910F91FF90EF90DF9052
:10256000CF90BF900C94750F002321F0812F9B2DED
:10257000937002C080E090E026960FB6F894DEBF1C
:102580000FBECDBFDF91CF911F910F91FF90EF90C4
:10259000DF90CF90BF900C94A30F812F002319F0F0
:1025A0000E94EC1D02C00E94541E26960FB6F8949D
:1025B000DEBF0FBECDBFDF91CF911F910F91FF9076
:1025C000EF90DF90CF90BF900C94D91E8B2D83702D
:1025D00009F07BC00111FBC1812F82958695877020
:1025E000880F880F912F9F70C92ED12CE12CF12CD0
:1025F000082E04C0CC0CDD1CEE1CFF1C0A94D2F784
:1026000014FF12C04FE050E060E070E004C0440FDF
:10261000551F661F771F8A95D2F7CB01BA016095C7
:1026200070958095909503C060E070E0CB012B2DF4
:10263000269526952370422F50E042305105D9F05F
:102640004330510569F16C297D298E299F2941303C
:10265000510551F126960FB6F894DEBF0FBECDBFDF
:10266000DF91CF911F910F91FF90EF90DF90CF906E
:10267000BF900C944C196C297D298E299F29269690
:102680000FB6F894DEBF0FBECDBFDF91CF911F9183
:102690000F91FF90EF90DF90CF90BF900C94661950
:1026A0000E944C19C701B60126960FB6F894DEBFFA
:1026B0000FBECDBFDF91CF911F910F91FF90EF9093
:1026C000DF90CF90BF900C943219002319F08B2D1E
:1026D000817001C08695882309F479C1812F829584
:1026E00086958770880F880F912F9F70C92ED12CE7
:1026F000E12CF12C082E04C0CC0CDD1CEE1CFF1CC0
:102700000A94D2F714FF12C04FE050E060E070E08E
:1027100004C0440F551F661F771F8A95D2F7CB015F
:10272000BA01609570958095909503C060E070E067
:10273000CB012B2D269526952370422F50E0423059
:102740005105D9F04330510569F16C297D298E2955
:102750009F294130510551F126960FB6F894DEBFFE
:102760000FBECDBFDF91CF911F910F91FF90EF90E2
:10277000DF90CF90BF900C94131A6C297D298E297D
:102780009F2926960FB6F894DEBF0FBECDBFDF910E
:10279000CF911F910F91FF90EF90DF90CF90BF905E
:1027A0000C94251A0E94131AC701B60126960FB67B
:1027B000F894DEBF0FBECDBFDF91CF911F910F9177
:1027C000FF90EF90DF90CF90BF900C94011A103FD4
:1027D000D1F128F480E4810F803250F0A0C0123F84
:1027E00009F462C008F44BC0133F09F472C097C0EB
:1027F000F12FF071FF2E8B2D8F71002351F00E946D
:102800009A19812FFF2019F08295807F68CE8F70F2
:1028100066CE0E94BB19812FFF2019F08295807F20
:1028200001C08F7026960FB6F894DEBF0FBECDBFE5
:10283000DF91CF911F910F91FF90EF90DF90CF909C
:10284000BF900C94BA110023B1F0253008F0BFC03E
:102850008B2D8F7126960FB6F894DEBF0FBECDBFBD
:10286000DF91CF911F910F91FF90EF90DF90CF906C
:10287000BF900C94E019263008F0A9C0E9CF0023DE
:10288000A9F08B2D8F7126960FB6F894DEBF0FBE80
:10289000CDBFDF91CF911F910F91FF90EF90DF900F
:1028A000CF90BF900C949A19002359F38B2D8F7100
:1028B00026960FB6F894DEBF0FBECDBFDF91CF9145
:1028C0001F910F91FF90EF90DF90CF90BF900C94ED
:1028D000BB19002399F08B2D8F7126960FB6F894B3
:1028E000DEBF0FBECDBFDF91CF911F910F91FF9043
:1028F000EF90DF90CF90BF900C94851926960FB67D
:10290000F894DEBF0FBECDBFDF91CF911F910F9125
:10291000FF90EF90DF90CF90BF900C948019002330
:10292000A9F0222309F4ADCF812F26960FB6F89493
:10293000DEBF0FBECDBFDF91CF911F910F91FF90F2
:10294000EF90DF90CF90BF900C941C11222309F4DC
:10295000ADCF812F26960FB6F894DEBF0FBECDBF48
:10296000DF91CF911F910F91FF90EF90DF90CF906B
:10297000BF900C9487114B2D4F70612FC6010E94A0
:10298000661D26960FB6F894DEBF0FBECDBFDF9151
:10299000CF911F910F91FF90EF90DF90CF90BF905C
:1029A0000C9480184B2D4F70612FC60126960FB6E0
:1029B000F894DEBF0FBECDBFDF91CF911F910F9175
:1029C000FF90EF90DF90CF90BF900C94691D2696FA
:1029D0000FB6F894DEBF0FBECDBFDF91CF911F9130
:1029E0000F91FF90EF90DF90CF90BF9008950E94DD
:1029F000701B0E943F1B0E94941B0E940B200E9490
:102A0000D91E80E090E00E94750F80E090E00C9469
:102A1000A30F0E94601B0C94F714CF93DF9300D098
:102A200000D01F92CDB7DEB70E94381A292F229509
:102A30002F7030E02C3031054CF42A303105C4F4CD
:102A4000225031092230310540F023C02C303105AD
:102A5000D1F02F303105B9F01CC0853A28F484300C
:102A6000B0F4823028F413C090E2980F983078F0D8
:102A7000883E30F4803E58F48450813A50F407C0C8
:102A8000803F39F404C093FB882780F903C081E0BC
:102A900001C080E00F900F900F900F900F90DF918A
:102AA000CF910895CF93DF9300D000D01F92CDB780
:102AB000DEB70F900F900F900F900F90DF91CF9196
:102AC0000895CF93DF9300D000D000D0CDB7DEB70C
:102AD00026960FB6F894DEBF0FBECDBFDF91CF9123
:102AE00008951F93CF93DF93C0919F0116E08091CB
:102AF000A001C81799F0D0E01C9FF0011D9FF00DB8
:102B00001124EF55FE4F4081518162817381848190
:102B100095810E9461152196C770E9CFDF91CF9111
:102B20001F9108954091D1015091D2016091D3013C
:102B30007091D4018091D5019091D6010C946115CA
:102B40008091D60182958F7009F054C08091D30195
:102B5000882309F44FC080919F01A091A00160914A
:102B6000D1017091D2014091D4015091D501B6E0CC
:102B70008A1709F43FC090E041155105C1F17F3F2C
:102B800011F46F3FA1F1B89FF001B99FF00D11242E
:102B9000EF55FE4F218172132AC02081621327C096
:102BA0002281211124C0238134812417350710F498
:102BB00021503109241B350B2C323140C0F42091B7
:102BC000D6012F7020612093D60126E0289FF001C6
:102BD000299FF00D1124EA55FE4F80818F7080618E
:102BE000808381ED91E00E94C1110C9471150196D2
:102BF0008770BECF0895BF92CF92DF92EF92FF927F
:102C00000F931F93CF93DF93CDB7DEB761970FB6C6
:102C1000F894DEBF0FBECDBF7C0185E0F701DE0179
:102C20001D9601900D928A95E1F7D7014C9111966E
:102C30005C9111971296DC90129713960D911C914E
:102C400014973091D1016091D2018091D40190917B
:102C5000D501009709F47FC16F3F19F43F3F09F494
:102C60007AC1B090D301BB2009F4CAC02091D6012B
:102C70000817190750F0F801E81BF90BCF01CC2415
:102C8000C3948C329140D0F009C080959095800F0C
:102C9000911FCC24C3948C32914080F0C12C207FB2
:102CA00009F0CCC0702F198B088B6D2D89890E947B
:102CB000521581ED91E00E94C111B6C0822F807F34
:102CC00009F047C0651314C0341312C0D11010C0EE
:102CD0002F7020612093D6010E94921581ED91E022
:102CE0000E94C1118091D601D70115968C932FC0F7
:102CF0000115110519F15F3F11F44F3FF9F0CD2C8B
:102D0000D1101CC080919F012091A00136E0821754
:102D100009F45CC090E0389FF001399FF00D112458
:102D2000EF55FE4F6181561306C06081461303C004
:102D30006281611103C001968770E9CFCD2CDD203F
:102D400009F429C18091D60181608093D601C12CFC
:102D500022C1651308C0341306C0D11004C080918D
:102D6000D601D701CCC04D875E87DF86702F198BC7
:102D7000088B6D2D89890E940D158823E9F1DD20CE
:102D8000D9F12091D601822F82958F7090E0029721
:102D900074F08091D1019091D20198878F83198628
:102DA0001B870A872C87CE0107960E94C11186E0F7
:102DB000F701A1EDB1E001900D928A95E1F70E9433
:102DC000A0150E949215CC24C394E5C0702F198BD6
:102DD000088B60E089890E94381A292F22952F706C
:102DE00030E0223031050CF0CAC09F7009F0C4C039
:102DF000805E883008F4CFC0C7010E94C111E3CFC4
:102E00000817190708F456C0F801E81BF90BCF01A1
:102E10008C32914008F456C0C12C702F198B088B4E
:102E20006D2D89890E945215E1EDF1E086E0DF0108
:102E30001D928A95E9F70E949215ADC0651314C0E2
:102E4000341312C0D11010C08091D601F7018583D0
:102E5000C7010E94C11186E0E1EDF1E0DF011D92A2
:102E60008A95E9F7CB2C97C04D875E87DF86702F58
:102E7000198B088B6D2D89890E940D15882309F403
:102E8000BBCFDD2009F4B8CF2091D601822F8295E7
:102E90008F7090E002970CF48ACF8091D1019091CD
:102EA000D2019A8389831B821D830C832E83CE01DA
:102EB00001967BCF80959095800F911F8C32914029
:102EC00008F0AACFCD2CDD2009F496CF65132EC0D3
:102ED00034132CC02091D60120FD1FC0822F829573
:102EE0008F70D9F0D70115962C9315978F3049F034
:102EF0008F5F982F9295907F822F8F70892B1596D8
:102F00008C93C7010E94C11186E0F701A1EDB1E0E9
:102F100001900D928A95E1F78ECF86E0F701A1ED41
:102F2000B1E001900D928A95E1F735C04D875E873B
:102F3000DF86702F198B088B6D2D89890E940D15E6
:102F4000811135CF8091D60181608093D601C70170
:102F50000E94C11120C0DD2009F44ECF4D875E874D
:102F6000DF86702F198B088B6D2D89890E940D15B6
:102F7000882309F441CF1BCF81113ACF0CC02430F4
:102F800031050CF039CF9F7009F432CFF7019581EC
:102F9000907F09F02DCF8C2D61960FB6F894DEBF8F
:102FA0000FBECDBFDF91CF911F910F91FF90EF909A
:102FB000DF90CF90BF9008951F93CF93DF93CDB74D
:102FC000DEB72C970FB6F894DEBF0FBECDBF4F8390
:102FD000588769877A878B879C87CE0107960E94DE
:102FE000FB15882369F08F8198852A853B85232BE3
:102FF000F1F19F3F09F063C08F3F09F060C037C017
:1030000086E0FE013796DE01119601900D928A95B9
:10301000E1F76F817885EA85FB85309741F17F3F45
:1030200011F46F3F21F12091A00130E0C901019618
:103030008770992740919F0150E08417950709F404
:1030400047C069837A83FD83EC8396E0929FD00129
:10305000939FB00D1124AF55BE4FFE0131960190E4
:103060000D929A95E1F78093A0010E94711516E0E8
:1030700080919F019091A0018917C1F1189FC00113
:1030800011248F559E4F0E94FB15882379F1E09102
:103090009F011E9FF0011124EF55FE4F4081518189
:1030A00062817381848195810E94611580919F0165
:1030B00090E001968770992780939F01D9CF4F8127
:1030C000588569857A858B859C850E946115CFCF4F
:1030D0000E9409151092A00110929F01E1EDF1E00C
:1030E00086E0DF011D928A95E9F7C1CF2C960FB6D5
:1030F000F894DEBF0FBECDBFDF91CF911F91089531
:10310000DF92EF92FF920F931F93CF93DF93FC0117
:10311000892B09F48AC0E12CF12CDD24D394EF0132
:1031200021968491853709F461C058F4843708F0FA
:103130004EC0843008F06AC08130D1F0823071F125
:1031400074C0883709F45DC050F4863709F455C05F
:10315000873709F06AC08E2D0E945D1B54C09CE722
:10316000980F903708F061C08F770E94871150C088
:103170008F010E5F1F4FFE01849190E2980F9830EF
:1031800050F48770FD2D01C0FF0F8A95EAF78F2F4D
:103190000E94631B14C00E941C1113C08F010E5F9C
:1031A0001F4FFE01C49180E28C0F883060F4C7701D
:1031B0008D2D01C0880FCA95EAF70E94691B0E94F5
:1031C000941BE80125C08C2F0E948711FACF9F0124
:1031D0002E5F3F4FFE01C491CC2369F08FE99FE041
:1031E0000197F1F700C00000C150F6CF9F012E5F9C
:1031F0003F4FFE01F490E9010BC00E944D1BE82EE9
:1032000007C00E94601B0E94941B02C00E941C11F8
:103210008F2D882341F0EFE9FFE03197F1F700C0EF
:1032200000008150F6CFFE017ACFDF91CF911F9140
:103230000F91FF90EF90DF90089560935702709385
:1032400058028093590290935A020C943A060895BA
:1032500060935B0270935C0280935D0290935E02C8
:103260000C942E1C0F931F9300915B0210915C0233
:1032700020915D0230915E02602B712B822B932B8B
:1032800060935B0270935C0280935D0290935E0298
:103290001F910F910C942E1C0F931F9300915B02B2
:1032A00010915C0220915D0230915E0260237123D7
:1032B0008223932360935B0270935C0280935D0290
:1032C00090935E021F910F910C942E1C0F931F93ED
:1032D00000915B0210915C0220915D0230915E02D0
:1032E000602771278227932760935B0270935C02AB
:1032F00080935D0290935E021F910F910C942E1C9F
:1033000060E070E0CB010C941D190F931F9341E016
:1033100050E060E070E08A019B0104C0000F111FC3
:10332000221F331F8A95D2F7C901B8011F910F914F
:103330000C941D190F931F9341E050E060E070E082
:1033400004C0440F551F661F771F8A95D2F78091DE
:10335000570290915802A0915902B0915A028A01E5
:103360009B01082B192B2A2B3B2BC901B8011F915C
:103370000F910C941D190F931F9341E050E060E0F2
:1033800070E004C0440F551F661F771F8A95D2F75F
:103390004095509560957095809157029091580294
:1033A000A0915902B0915A028A019B010823192366
:1033B0002A233B23C901B8011F910F910C941D19B9
:1033C0000F931F9341E050E060E070E004C0440FB1
:1033D000551F661F771F8A95D2F7809157029091EB
:1033E0005802A0915902B0915A028A019B01082704
:1033F00019272A273B27C901B8011F910F910C9467
:103400001D190F931F93009157021091580220919C
:10341000590230915A02602B712B822B932B1F91F2
:103420000F910C941D190F931F9300915702109147
:1034300058022091590230915A026023712382234D
:1034400093231F910F910C941D190F931F930091BB
:103450005702109158022091590230915A02602768
:103460007127822793271F910F910C941D1908959E
:103470008F929F92AF92BF92DF92EF92FF920F9343
:103480001F93CF93DF9300D000D01F92CDB7DEB74C
:103490008A016623C9F180905B0290905C02A09043
:1034A0005D02B0905E028091570290915802A09107
:1034B0005902B0915A02882A992AAA2ABB2A8FE176
:1034C000E82EF12CD501C4010E2C04C0B695A795A9
:1034D000979587950A94D2F780FF07C0DE2CB80134
:1034E0008E2D0E943C1D019729F481E0E81AF10815
:1034F00048F7D12C80E1189FF0011124E00FF11D55
:10350000E952FE4FD08209C080E1189FF0011124DA
:10351000E40FF11DE952FE4FD08009831A836981BF
:103520007A818D2D0E943C1D0F900F900F900F906F
:103530000F90DF91CF911F910F91FF90EF90DF904F
:10354000BF90AF909F908F90089590910A0199231A
:1035500021F090910B01911109C020910C01309143
:103560000D01F90132969FEF40E030C0982F9695FB
:10357000969596959F31A0F4E0910C01F0910D0184
:10358000E90FF11D877021E030E0A90102C0440F6E
:10359000551F8A95E2F7CA019181892B818308958D
:1035A0009091840290FF23C01F928F938CE094E04F
:1035B0009F938F930E9431060F900F900F900F9062
:1035C00008959F3F39F04F5F4E3141F051915813AC
:1035D000F8CF0DC05111F7CF942FF5CF9F3F39F0A1
:1035E000F901E90FF11D97FDFA9582830895089579
:1035F00090910A01992321F090910B01911109C03A
:1036000020910C0130910D01F9013296205E3F4F5F
:1036100030C0982F9695969596959F31A8F4E09195
:103620000C01F0910D01E90FF11D877021E030E0F0
:10363000A90102C0440F551F8A95E2F7CA0180957F
:1036400091818923818308959091840290FF16C00F
:103650001F928F938EEE93E09F938F930E9431067B
:103660000F900F900F900F9008953196E217F30787
:1036700029F090819813F9CF1082F7CF089581E057
:1036800090E0E0910C01F0910D01E80FF91F10821C
:10369000019680329105A9F70895809183020895DB
:1036A00090918302892B8093830208958095909155
:1036B000830289238093830208958093830208956F
:1036C00010928302089590918202892B8093820246
:1036D00008958095909182028923809382020895B3
:1036E000109282020895809361020E94A51C90931B
:1036F000600280935F02089510926102109260024E
:1037000010925F02089580910C0190910D01FC01CF
:1037100031969C01205E3F4F80E0919191118F5F27
:10372000E217F307D1F70895E0910C01F0910D0134
:10373000809183028083E0910C01F0910D019081D2
:1037400080918202892B8083809161028823D9F144
:103750000E94A51C20915F0230916002821793079E
:1037600048F00E94A51C20915F0230916002821BEC
:10377000930B0AC00E94A51C20915F023091600249
:1037800020953095820F931F8C32914070F080917C
:10379000840280FF08C08AE294E09F938F930E9486
:1037A00031060F900F900E947C1BE0910C01F0916C
:1037B0000D01908180916102892B80830E94831B7F
:1037C00081110E947C1B80910C0190910D010C9441
:1037D000210F909339018093380108958295982F95
:1037E0009C7C392F36953695282F237344E0249FEF
:1037F000C0011124932F982B292F2A7A2695892FDF
:103800008575880F822B08951F93CF93DF931F92A6
:10381000CDB7DEB799830E94EE1B182F9981892FAF
:103820000E94EE1B212F30E0322F2227A901482BC6
:10383000CA010F90DF91CF911F9108950895CF9302
:10384000DF9300D000D01F92CDB7DEB70F900F905E
:103850000F900F900F90DF91CF91089508950C94E1
:10386000A21080919902843021F11092850220E407
:1038700088E190E00FB6F894A895809360000FBEA1
:103880002093600083B7817F846083BF83B78160AA
:1038900083BF7894889583B78E7F83BF0FB6F894E3
:1038A000A89580916000886180936000109260000C
:1038B0000FBE0895CF930E94DA100E946E060E94F8
:1038C000DB10C0E08C2F0E943E07892B29F4CF5FCC
:1038D000C830C1F780E001C081E0CF9108950E9417
:1038E000A4100C9409151F920F920FB60F92112479
:1038F0008F939F93AF93BF9380918502811113C0E3
:103900008091860290918702A0918802B0918902ED
:103910004196A11DB11D8093860290938702A093CA
:103920008802B0938902BF91AF919F918F910F90C0
:103930000FBE0F901F90189582E084BD93E095BD57
:103940009AEF97BD80936E0008952FB7F8948091F9
:10395000860290918702A0918802B09189022FBFC0
:1039600008952FB7F8946091860270918702809134
:103970008802909189022FBF0895CF92DF92EF9233
:10398000FF920F931F932FB7F894409186025091A6
:10399000870260918802709189022FBF6A017B01C2
:1039A000EE24FF248C0120E030E0C016D106E206B0
:1039B000F30610F4415051099A01281B390BC90133
:1039C0001F910F91FF90EF90DF90CF9008951F927D
:1039D0000F920FB60F9211248F939F93AF93BF93C3
:1039E0008091860290918702A0918802B09189020D
:1039F0000196A11DB11D8093860290938702A0932A
:103A00008802B0938902BF91AF919F918F910F90DF
:103A10000FBE0F901F9018950E942E0CF8942FEF58
:103A200087EA91E6215080409040E1F700C0000015
:103A300087E090EBDC018093A2029093A302A09315
:103A4000A402B093A5029CE088E10FB6F894A89573
:103A5000809360000FBE90936000FFCF20E1929FA3
:103A6000F0011124E80FF11DE052FF4F9491892FCE
:103A70008F7092959F700895CF93C82FCB010E94AD
:103A80002E1D282F30E080E1989FA0011124422BA9
:103A9000532B4038510519F480E090E015C0977021
:103AA000E92FF0E088E0C89FE00DF11D112484E0CB
:103AB000EE0FFF1F8A95E1F7E20FF31FEE0FFF1FD6
:103AC000E050F84985919491CF91089580E090E07D
:103AD0000895089580918C0280FF0BC060911101C0
:103AE00085E0689FB0011124759567957595679578
:103AF0002BC081FF09C06091110185E0689FB00172
:103B000011247595679520C082FF07C0609111014F
:103B100085E0689FB001112417C090918D02992310
:103B2000D1F060911001961788F72091110185E07E
:103B3000289F90011124929FA001939F500D112462
:103B400070E0CA010E9442256038710540F4611599
:103B5000710539F002C065E070E0862F08958FE7A7
:103B6000089581E0089580918C0280FF08C06091E3
:103B70000F0170E0759567957595679521C081FF78
:103B800006C060910F0170E07595679519C082FFBE
:103B900004C060910F0170E010C090918D029923D4
:103BA000C1F060910E019617A0F780910F01899FD7
:103BB000C001112470E00E9442256038710528F48C
:103BC0006115710521F0862F08958FE7089581E032
:103BD000089561E070E0F4CF803F21F40E946A1DF7
:103BE000819504C0813F29F40E946A1D8093900250
:103BF0000895823F21F40E946A1D819504C0833F8D
:103C000029F40E946A1D80938F020895893F19F458
:103C10000E94B31D05C08A3F31F40E94B31D8195F7
:103C20008093910208958B3F21F40E94B31D8195EA
:103C300004C08C3F29F40E94B31D80939202089522
:103C4000843F21F480918E02816017C0853F21F46A
:103C500080918E02826011C0863F21F480918E0295
:103C600084600BC0873F21F480918E02886005C07C
:103C7000883F31F480918E02806180938E02089596
:103C80008D3F21F480918C0281600BC08E3F21F426
:103C900080918C02826005C08F3F29F480918C0254
:103CA000846080938C020895803F39F48091900263
:103CB00087FF6CC01092900269C0813F29F4809107
:103CC00090021816BCF362C090918F02823F29F4D3
:103CD00097FF5CC010928F0259C0833F19F41916E8
:103CE000CCF354C0893F41F48091910218160CF036
:103CF0004DC0109291024AC08A3F29F480919102EE
:103D000087FF44C0F6CF8B3F39F48091920287FF42
:103D10003DC0109292023AC08C3F29F480919202E9
:103D20001816BCF333C0843F21F480918E028E7F3D
:103D300017C0853F21F480918E028D7F11C0863F90
:103D400021F480918E028B7F0BC0873F21F48091FC
:103D50008E02877F05C0883F31F480918E028F7E6E
:103D600080938E0213C08D3F21F480918C028E7F50
:103D70000BC08E3F21F480918C028D7F05C08F3F58
:103D800029F480918C028B7F80938C0280918F022A
:103D900081110EC08091900281110AC08091910220
:103DA000811106C080919202811102C010928D0291
:103DB00008958091840283FF7EC083E694E00E9490
:103DC000980580918E021F928F938EE594E09F93C9
:103DD0008F930E9431068CE594E00E9498058091B3
:103DE0008F02282F082E000C330B3F938F9389E509
:103DF00094E09F938F930E94310687E594E00E94A0
:103E0000980580919002282F082E000C330B3F93C9
:103E10008F9384E594E09F938F930E94310682E50F
:103E200094E00E94980580919102282F082E000CA2
:103E3000330B3F938F938FE494E09F938F930E9473
:103E400031068DE494E00E94980580919202282F1B
:103E5000082E000C330B3F938F938AE494E09F93DA
:103E60008F930E94310687E494E00E949805809128
:103E70008D021F928F9384E494E09F938F930E940E
:103E8000310682E494E00E94980580918C021F9292
:103E90008F938FE394E09F938F930E9431068CE37E
:103EA00094E00E9498058DB79EB74C960FB6F89493
:103EB0009EBF0FBE8DBF8EE892E00E946A0F0E94E7
:103EC000A51C90938B0280938A0208951F93CF9331
:103ED000DF9380918A0290918B020E94BD1CAC01FD
:103EE00090918D02992321F02091120130E006C0BB
:103EF000209113018AE0289F900111244217530753
:103F000008F485C080918F02C0919002D0919102F7
:103F100010919202811107C0C11175C0D11173C0F7
:103F2000111171C074C09F3F19F09F5F90938D0273
:103F3000181624F40E946A1D80938F0280918F02CC
:103F400087FF05C00E946A1D819580938F021C1611
:103F500024F40E946A1D809390028091900287FF52
:103F600005C00E946A1D81958093900260918F0226
:103F7000662331F1C0919002CC2311F1062E000C82
:103F8000770B880B990B0E943D2423E333E343E333
:103F90005FE30E94A1240E94052460938F026C2F8E
:103FA000CC0F770B880B990B0E943D2423E333E35E
:103FB00043E35FE30E94A1240E94052460939002E2
:103FC0001D1624F40E94B31D8093910280919102EA
:103FD00087FF05C00E94B31D819580939102111641
:103FE00024F40E94B31D809392028091920287FF75
:103FF00005C00E94B31D819580939202DF91CF91FD
:104000001F910C94D91E9F3F09F08FCF97CFDF915E
:10401000CF911F910895EEE8F2E085E0DF011D9257
:104020008A95E9F710928D0210928C02089586E825
:1040300096E00E9498051F9281E08F931F9285E081
:104040008F9388E396E09F938F930E9431060F90A1
:104050000F900F900F900F900F9008958330E9F11B
:1040600028F4813061F0823009F10895853009F437
:1040700062C008F449C0863009F474C00895809184
:104080001301262F30E0280F311D2F3F310524F476
:10409000680F6093130103C08FEF80931301809129
:1040A00013011F928F9381E795E072C080911201F6
:1040B000262F30E0280F311D2F3F310524F4680FE3
:1040C0006093120103C08FEF80931201809112015F
:1040D0001F928F938FE595E05BC080911101262F91
:1040E00030E0280F311D2F3F310524F4680F609315
:1040F000110103C08FEF80931101809111011F9274
:104100008F938CE495E044C080911001262F30E01D
:10411000280F311D2F3F310524F4680F60931001E3
:1041200003C08FEF80931001809110011F928F9335
:1041300087E395E02DC080910F01262F30E0280FF6
:10414000311D2F3F310524F4680F60930F0103C028
:104150008FEF80930F0180910F011F928F938EE15B
:1041600095E016C080910E01262F30E0280F311DFA
:104170002F3F310524F4680F60930E0103C08FEFC9
:1041800080930E0180910E011F928F9383E095E042
:104190009F938F930E9431060F900F900F900F9076
:1041A0000895833081F128F4813059F08230D1F0C4
:1041B0000895853009F449C0B8F1863009F456C035
:1041C000089580911301681720F4861B80931301D2
:1041D00002C010921301809113011F928F9384EFFC
:1041E00094E054C080911201681720F4861B8093DC
:1041F000120102C010921201809112011F928F933E
:1042000082EE94E043C080911101681720F4861B70
:104210008093110102C010921101809111011F922F
:104220008F938FEC94E032C080911001681720F4D6
:10423000861B8093100102C0109210018091100122
:104240001F928F938AEB94E021C080910F01681731
:1042500020F4861B80930F0102C010920F01809101
:104260000F011F928F9381EA94E010C080910E019C
:10427000681720F4861B80930E0102C010920E0175
:1042800080910E011F928F9386E894E09F938F9305
:104290000E9431060F900F900F900F900895CF93CA
:1042A000C82F1F928F938BE897E09F938F930E9464
:1042B000310681E090E0A0E0B0E0BC01CD0104C097
:1042C000660F771F881F991FCA95D2F70E94281979
:1042D0000F900F900F900F90CF910C940915CF93E2
:1042E0008732A8F58E3108F02BC1803109F49FC0C8
:1042F000F8F4873009F464C0A8F4863009F024C1CA
:1043000080918402817F8E7F8093840280E997E090
:104310000E94980581E89AE00E94980581E08093C8
:1043200094024CC08B30F1F18E3009F46CC00CC19A
:10433000863109F4B0C020F4813109F4EDC004C124
:10434000893109F491C08B3109F449C0FDC088332B
:1043500049F150F4893209F4F1C0853309F4EEC013
:10436000873209F0F1C0EAC0833409F4E7C028F4C9
:104370008A3308F4E9C08953E4C0883409F0E4C002
:104380000E94091580E79AE00E9498052FEF83EDBF
:1043900090E3215080409040E1F700C000000E946F
:1043A0000C1D0CC087EB97E05CC087E59AE00E948B
:1043B000980580918402816080938402C1E0C9C025
:1043C00080918402C82FC17080FFEFCF83E69AE00E
:1043D0000E94980580918402817F8E7F3DC09091DC
:1043E000840291FBCC27C0F981E0C827892FC0FB4C
:1043F00081F980938402CC2319F08AE49AE027C0E3
:104400008CE39AE02EC09091840292FBCC27C0F9F5
:1044100081E0C827892FC0FB82F980938402CC23D6
:1044200019F08DE29AE013C08DE19AE01AC09091E4
:10443000840293FBCC27C0F981E0C827892FC0FBF9
:1044400083F980938402CC2351F081E19AE00E94A9
:104450009805809184028160809384027AC084E010
:104460009AE00E949805AACF85EF99E00E949805EE
:104470008CEC99E00E9498058AE899E00E949805E2
:104480008DE599E00E94980583E199E00E949805E6
:1044900085EE98E0E6CF87ED98E00E9498050E94AF
:1044A000150F1F928F938DEB98E09F938F930E942F
:1044B000310680910A011F928F9386EA98E09F93BC
:1044C0008F930E943106809187011F928F9383E919
:1044D00098E09F938F930E94310680910B011F9269
:1044E0008F9380E898E09F938F930E9431060E94FB
:1044F000B11C9F938F937F936F9389E698E09F936E
:104500008F930E9431068DB79EB746960FB6F894EA
:104510009EBF0FBE8DBF52CF0E940915C0910B01E7
:1045200081E0C827C0930B01CC2329F08FE598E0E8
:104530000E9498050EC084E598E093CF80E001C00A
:104540008D510E944F213ACF82E598E00E94980554
:10455000C0E08C2FCF91089580E0089580E0089509
:10456000CF93C82F80919402813071F020F0823077
:1045700009F44BC042C1E0910C01F0910D01808122
:10458000823209F03CC107C0E0910C01F0910D01AD
:104590008081823261F48C2F0E94AC22811104C090
:1045A0008C2F0E946F212FC081E090E02CC08C2FB7
:1045B0000E94AE22811126C0C431E1F070F4CB30EC
:1045C00081F0C031D1F40E94172083E897E00E9467
:1045D000980582E08093940215C0C93259F0C8331F
:1045E00061F480E997E00E94980587E897E00E94CF
:1045F000980508C01092940204C181E897E00E94D7
:104600009805FFC081E08170FEC0C43228F5CE312C
:1046100008F0C1C0CB30A1F1D0F4C73009F0D3C04D
:104620008EE18093130182E3809312018AE08093EC
:10463000110184E18093100188E080930F0188E2EA
:1046400080930E0187E296E00E949805BFC0C331B7
:1046500049F1C431C1F0B7C0CB3409F4A9C028F482
:10466000C93289F0C83361F0AEC0C13509F49EC0CB
:10467000C23509F499C0CE3409F0A5C06AE09EC0E5
:104680000E941720A3C080919302882319F01092F2
:1046900093029CC084E396E00E94980581E0809399
:1046A0009402B1C08EE096E00E9498058CEF95E0F0
:1046B0000E949805809113011F928F9389EF95E0D6
:1046C0009F938F930E94310687EF95E00E94980593
:1046D00085EE95E00E949805809112011F928F93BC
:1046E00082EE95E09F938F930E94310680EE95E0D5
:1046F0000E94980581ED95E00E9498058091110136
:104700001F928F938EEC95E09F938F930E943106BA
:104710008CEC95E00E9498058BEB95E00E94980543
:10472000809110011F928F9388EB95E09F938F9358
:104730000E94310686EB95E00E94980581EA95E09B
:104740000E94980580910F011F928F938EE995E04A
:104750009F938F930E9431068CE995E00E94980503
:1047600085E895E00E94980580910E011F928F9335
:1047700082E895E09F938F930E94310680E895E050
:104780000E9498058DB79EB748960FB6F8949EBFC5
:104790000FBE8DBF1BC0CE51EC2FF0E0E25DFE4F8F
:1047A00080818093930212C061E003C061E006C083
:1047B0006AE0809193020E942E2008C080919302AB
:1047C0000E94D12003C085E296E013C0809193023D
:1047D000882369F01F928F938FE196E09F938F93C8
:1047E0000E9431060F900F900F900F9004C08CE143
:1047F00096E00E94980581E006C01092940280E045
:1048000002C080E000CFCF9108950E940C246894EC
:10481000B1110C949B2408950E94802488F09F5726
:1048200098F0B92F9927B751B0F0E1F0660F771FD4
:10483000881F991F1AF0BA95C9F714C0B13091F0CA
:104840000E949A24B1E008950C949A24672F782F3F
:104850008827B85F39F0B93FCCF38695779567958F
:10486000B395D9F73EF490958095709561957F4FFB
:104870008F4F9F4F0895E89409C097FB3EF49095A1
:104880008095709561957F4F8F4F9F4F9923A9F029
:10489000F92F96E9BB279395F695879577956795B8
:1048A000B795F111F8CFFAF4BB0F11F460FF1BC0FC
:1048B0006F5F7F4F8F4F9F4F16C0882311F096E98F
:1048C00011C0772321F09EE8872F762F05C066233D
:1048D00071F096E8862F70E060E02AF09A95660FF6
:1048E000771F881FDAF7880F9695879597F90895AF
:1048F00057FD9058440F551F59F05F3F71F0479591
:10490000880F97FB991F61F09F3F79F08795089575
:10491000121613061406551FF2CF4695F1DF08C094
:10492000161617061806991FF1CF869571056105B1
:1049300008940895E894BB2766277727CB0197F959
:1049400008950E94B4240C9425250E94172538F060
:104950000E941E2520F0952311F00C940E250C9436
:10496000142511240C949B240E94782470F3959FA5
:10497000C1F3950F50E0551F629FF001729FBB2756
:10498000F00DB11D639FAA27F00DB11DAA1F649FF2
:104990006627B00DA11D661F829F2227B00DA11DA5
:1049A000621F739FB00DA11D621F839FA00D611D2B
:1049B000221F749F3327A00D611D231F849F600D4C
:1049C000211D822F762F6A2F11249F5750409AF075
:1049D000F1F088234AF0EE0FFF1FBB1F661F771F01
:1049E000881F91505040A9F79E3F510580F00C94CC
:1049F0000E250C949B245F3FE4F3983ED4F38695F8
:104A000077956795B795F795E7959F5FC1F7FE2B6B
:104A1000880F911D9695879597F9089597F99F6747
:104A200080E870E060E008959FEF80EC0895002436
:104A30000A941616170618060906089500240A9403
:104A400012161306140605060895092E0394000C89
:104A500011F4882352F0BB0F40F4BF2B11F460FF18
:104A600004C06F5F7F4F8F4F9F4F0895991B79E070
:104A700004C0991F961708F0961B881F7A95C9F7EE
:104A80008095089597FB072E16F4009407D077FDC4
:104A900009D00E945C2507FC05D03EF490958195D5
:104AA0009F4F0895709561957F4F0895EE0FFF1FFA
:104AB0000590F491E02D0994AA1BBB1B51E107C09E
:104AC000AA1FBB1FA617B70710F0A61BB70B881F9E
:104AD000991F5A95A9F780959095BC01CD0108952D
:044AE000F894FFCF78
:104AE400510742081F08EB07B707010162022808B3
:104AF400140A321E404D3622394D030003CA02A85F
:104B0400026F02E201FB0114022D024D02000102B8
:084B140003040506070809006F
:106800000000000000000000040005000600070072
:10681000080009000A000B000C000D000E000F001C
:1068200010001100120013001400150016001700CC
:10683000180019001A001B001C001D001E001F007C
:10684000200021002200230024002500260027002C
:10685000280000002A002B002C002D002E002F0005
:1068600030003100000033003400290036003700CA
:106870003800E00000000000000000000000000000
:106880000000000000000000000000000000000008
:1068900000004900000000004C00000000004F0014
:1068A00050005100520000000000000000000000F5
:1068B00000000000000000000000000000000000D8
:1068C00000000000000000000000000000000000C8
:1068D00000000000000000000000000000000000B8
:1068E00000000000000000000000000000000000A8
:1068F000E000C2A2E200E300E400D2A2E600F1A3BD
:106900000000000000000000040005000600070071
:10691000080009000A000B000C000D000E000F001B
:1069200010001100120013001400150016001700CB
:10693000180019001A001B001C001D001E001F007B
:10694000200021002200230024002500260027002B
:10695000280000002A002B002C002D002E002F0004
:1069600030003100000033003400350036003700BD
:106970003800E000000000000000000000000000FF
:106980000000000000000000000000000000000007
:1069900000004900000000004C00000000004F0013
:1069A00050005100520000000000000000000000F4
:1069B00000000000000000000000000000000000D7
:1069C00000000000000000000000000000000000C7
:1069D00000000000000000000000000000000000B7
:1069E00000000000000000000000000000000000A7
:1069F000E000E100E200E300E400E500E600F1A4CD
:106A00000000000000000000010001000100010082
:106A1000010001000100010001000100010001006E
:106A2000010001000100010001000100010001005E
:106A3000010001000100010001000100010001004E
:106A4000010001000100010001000100010001003E
:106A5000010000000100010001000100010001002F
:106A600001000100000001000100350001000100EB
:106A70000100010000000000000000000000000014
:106A80000000000000000000000000000000000006
:106A900000000100000000000100000000000100F3
:106AA00001000100010000000000000000000000E3
:106AB00000000000000000000000000000000000D6
:106AC00000000000000000000000000000000000C6
:106AD00000000000000000000000000000000000B6
:106AE00000000000000000000000000000000000A6
:106AF000010001000100010001000100010001008E
:106B00000000000000000000EA4401000100E2442F
:106B10000100010001000100460001004A004B0095
:106B20000100010047004800028A0100E944010019
:106B30000100010001000100010001003A003B00DA
:106B40003C003D003E003F00400041004200430049
:106B5000010000000100390001004400450001006F
:106B60000100010000000100010035004D004E0051
:106B70000100010000000000000000000000000013
:106B80000000000000000000000000000000000005
:106B900000000100000000000100000000004D00A6
:106BA0004A004E004B000000000000000000000002
:106BB00000000000000000000000000000000000D5
:106BC00000000000000000000000000000000000C5
:106BD00000000000000000000000000000000000B5
:106BE00000000000000000000000000000000000A5
:106BF0000100010001000100650001000100F1A396
:106C00000000000000000000EA4401000100E2442E
:106C10000100010001000100460001004A004B0094
:106C20000100010047004800028A0100E944010018
:106C30000100010001000100010001003A003B00D9
:106C40003C003D003E003F00400041004200430048
:106C5000010000000100390001004400450001006E
:106C60000100010000000100010029004D004E005C
:106C70000100010000000000000000000000000012
:106C80000000000000000000000000000000000004
:106C900000000100000000000100000000004D00A5
:106CA0004A004E004B000000000000000000000001
:106CB00000000000000000000000000000000000D4
:106CC00000000000000000000000000000000000C4
:106CD00000000000000000000000000000000000B4
:106CE00000000000000000000000000000000000A4
:106CF0000100010001000100650001000100F1A494
:00000001FF
